:020000040800F2
:100000000005002001010008250100082701000863
:10001000290100082B0100082D0100080000000044
:100020000000000000000000000000002F01000898
:10003000310100080000000033010008350100080C
:1000400037010008370100083701000837010008B0
:1000500037010008370100083701000837010008A0
:100060003701000837010008370100083701000890
:100070003701000837010008370100083701000880
:100080003701000837010008370100083701000870
:100090003701000837010008370100083701000860
:1000A0003701000837010008370100083701000850
:1000B0003701000837010008370100083701000840
:1000C0003701000837010008370100083701000830
:1000D0003701000837010008370100083701000820
:1000E000370100083701000837010008DFF80CD09D
:1000F00000F02CF80048004791010008000500209E
:100100000D488047DFF83400016841F4E0210160C8
:10011000BFF34F8FDFF82800DFF8281001600A488E
:1001200000477047FEE7FEE7FEE7FEE7FEE7FEE773
:10013000FEE7FEE7FEE7FEE72301000824ED00E00E
:100140000CED00E00003FA05ED000008064C074D39
:1001500006E0E06840F0010394E807009847103497
:10016000AC42F6D3FFF7C6FF2002000830020008B9
:1001700002E008C8121F08C1002AFAD17047704770
:10018000002001E001C1121F002AFBD170470000CE
:10019000002406E0204600F029F8044941F8240034
:1001A000641C402CF6DB00BFFEE7000000000020CE
:1001B0004FF000024FF0000308B401B400FB02F05E
:1001C00000F03F0031F9103001BC02B4064931F9AA
:1001D00012C002BC0CFB03FC08BC634402F1010228
:1001E000402AE9D1184670473002000800B54DF8A2
:1001F000048D80460849FFF7DBFF01B440460749FC
:10020000FFF7D6FF02BC81FB0112C0FB00121046B3
:100210005DF8048B00BD704730030008B002000891
:10022000B003000800000020000500008001000865
:10023000A3087303B008B30B6F066205ED098509C7
:1002400035066107450913087A070708C1075108F1
:10025000D408F906F106F409D4081B05E407A20B3B
:10026000F7060604760ACB0B0904FC04520DAD090F
:10027000B5011C08B40EDC0591012D0C770D0902A7
:100280002304460FCB0914008608D20F2F0508015E
:10029000D40C790DAB017C042C0F5509B800D008A3
:1002A000B10E53057A020E0CF70B2B03BE05FA0CA8
:1002B000FF7F627F8A7D7D7A4276E3706E6AF262AA
:1002C000825A34511D47573CFC302825F9188C0CB4
:1002D000000074F307E7D8DA04CFA9C3E3B8CCAEC3
:1002E0007EA50E9D92951D8FBE89838576829E8008
:1002F00000809E8076828385BE891D8F92950E9D9B
:100300007EA5CCAEE3B8A9C304CFD8DA07E774F36F
:1003100000008C0CF9182825FC30573C1D4734513F
:10032000825AF2626E6AE37042767D7A8A7D627FDB
:1003300000008C0CF9182825FC30573C1D4734511F
:10034000825AF2626E6AE37042767D7A8A7D627FBB
:10035000FF7F627F8A7D7D7A4276E3706E6AF26209
:10036000825A34511D47573CFC302825F9188C0C13
:10037000000074F307E7D8DA04CFA9C3E3B8CCAE22
:100380007EA50E9D92951D8FBE89838576829E8067
:1003900000809E8076828385BE891D8F92950E9DFA
:1003A0007EA5CCAEE3B8A9C304CFD8DA07E774F3CF
:04000005080000ED02
:00000001FF
